:100000000EC01DC01CC01BC01AC019C018C017C02C
:1000100016C015C014C013C012C011C010C01124E6
:100020001FBECFE5D1E0DEBFCDBF10E0A0E6B0E05F
:1000300001C01D92A236B107E1F77CD0F7C0E0CF36
:10004000FC018081562F5095852380838CEC90E0B5
:100050000197F1F7242F332727FD309520FF03C0A8
:100060008081862B02C08081852380838CEC90E088
:100070000197F1F721FF03C08081862B02C08081A8
:10008000852380838CEC90E00197F1F722FF03C079
:100090008081862B02C08081852380838CEC90E058
:1000A0000197F1F723FF03C08081862B02C0808176
:1000B000852380838CEC90E00197F1F724FF03C047
:1000C0008081862B02C08081852380838CEC90E028
:1000D0000197F1F725FF03C08081862B02C0808144
:1000E000852380838CEC90E00197F1F726FF03C015
:1000F0008081862B02C08081852380838CEC90E0F8
:100100000197F1F747FF04C08081862B808303C0ED
:100110008081582350832CEC30E0C9010197F1F71E
:100120008081862B8083C9010197F1F7C90101976E
:10013000F1F70895CF92DF92EF92FF920F931F9302
:1001400080E886BD16BC8FE080BF84E089BFC09A7E
:10015000B89A82E087B987E886B988E390E061E0E1
:1001600043E56EDFCC24C39484E0D82EEE24FF2434
:10017000870120E030E0369A3699FECF84B195B100
:10018000A0E0B0E0E80EF91E0A1F1B1F2F5F3F4FD3
:100190002430310581F780916000882319F580EBC8
:1001A000E81684E0F80680E0080780E01807D0F43D
:1001B000C09260000FB407FC09C0809161008823E1
:1001C00029F488E390E061E046E43ADF0FB407FCED
:1001D00004C080916100882329F088E390E061E009
:1001E00043E52EDF80916000882379F08DEDE816DD
:1001F00085E0F80680E0080780E0180730F01FBCB3
:10020000D8BE109260001092610008B602FEAECF18
:10021000D8BE80916100882309F0A8CF88E390E0E0
:1002200061E04FE40DDFC0926100A0CFF894FFCFF2
:00000001FF
